:100000000C94C0000C94DD000C94DD000C94DD0019
:100010000C94DD000C94DD000C94DD000C94DD00EC
:100020000C94DD000C94310A0C94B1080C94040A71
:100030000C947D090C94AA090C9484080C94500922
:100040000C9425080C94DD000C94730D0C94DD00C9
:100050000C94290D0C942B010C94DD000C94DD0004
:100060000C94D7090C94E50A0C945E0A0C948B0A44
:100070000C94B80A0C9423090C94980D0C94DD0090
:100080000C944E0D0C94DD000C94DD002F65727203
:100090006F722F6D73676C656E6774682F002F65C4
:1000A00072726F722F74797065746167322F002FCE
:1000B0006572726F722F74797065746167332F0087
:1000C0002F6572726F722F74797065746167342F47
:1000D000002F6572726F722F6D736773697A652F67
:1000E000002F6572726F722F636865636B73756D35
:1000F0000000000100080020004000800000010016
:10010000040000010008004000000100043031320A
:1001100033343536373839414243444546002F7031
:10012000776D002F6F7574002F696E30002F696E28
:1001300031002F696E32002F696E33002F696E34E3
:10014000002F696E35002F696E36002F696E3700FB
:100150002F61646330002F61646331002F61646339
:1001600032002F61646333002F61646334002F61B8
:10017000646335002F61646336002F616463370068
:1001800011241FBECFEFD0E1DEBFCDBF11E0A0E054
:10019000B1E0EAE6F7E200E00BBF02C007900D9283
:1001A000A030B107D9F715E0A0E0B1E001C01D9281
:1001B000A830B107E1F70C9486100C94000096B1BA
:1001C000987F982B96B9089527B12F73992736E019
:1001D000880F991F3A95E1F7282B27B90895379A88
:1001E000359886E00E94DF0081E00E94E4003D989F
:1001F000339A1092A5047894089533983798089507
:1002000097B1907E8F71982B97B90895349A369A4A
:10021000089586B199278074907008951092A5046E
:1002200097B1907E8F71982B97B9349A369A3699F8
:10023000FECF84B1282F332785B19927982F88279F
:10024000822B932B08950E940E0196958795969583
:100250008795992708951F920F920FB60F92112438
:100260008F938FEF8093A5048F910F900FBE0F9007
:100270001F9018950E94790B40E052EC61E070E00D
:1002800080E00E94120B0895992781309105A1F01A
:10029000823091051CF4892B21F032C0029729F19C
:1002A0002FC080E00E94AD0B6CE20E94200E80E027
:1002B0000E94AD0B69E62EC080E00E94AD0B6CE29F
:1002C0000E94200E80E00E94AD0B69E60E94200E85
:1002D00080E00E94AD0B69E60E94200E80E00E9443
:1002E000AD0B60E00E94200E089580E00E94AD0BEF
:1002F0006CE20E94200E80E00E94AD0B63E70AC012
:1003000080E00E94AD0B6CE20E94200E80E00E9413
:10031000AD0B6EE40E94200E80E00E94AD0B60E009
:10032000DBCF0F931F93CF93DF93EC0100E0FE012F
:100330002196149180E00E94AD0B612F0E94200E47
:100340000F5F1123A1F7802F992783709070892B5D
:1003500069F080E00E94AD0B60E00E94200E0F5F0C
:10036000802F992783709070892B99F7DF91CF9117
:100370001F910F9108951F93CF93DF93EC01162FD8
:1003800080E00E94AD0B6EEB0E94200E20E0FE018B
:100390008491882329F02F5FFE01E20FF11DF8CF31
:1003A0002F5F822F992783709070892B11F02C7FFB
:1003B0002C5F120F80E00E94AD0B612F0E94200E77
:1003C000DF91CF911F9108950F931F93CF93DF93E8
:1003D000EC0100E0199180E00E94AD0B612F0E94BA
:1003E000200E0F5F1123B1F7802F99278370907033
:1003F000892B69F080E00E94AD0B60E00E94200E26
:100400000F5F802F992783709070892B99F7DF9168
:10041000CF911F910F9108950F931F93CF93DF9367
:1004200000E012E008C080E00E94AD0BBE010E9417
:100430000E0E080F1F5FC12FDD2780E00E94AD0B5D
:10044000FC0184819581C817D90768F380E00E9478
:10045000AD0B602F0E94200EDF91CF911F910F9165
:1004600008950F931F93CF93DF938C01EB0160E00E
:10047000FE018491882329F06F5FFE01E60FF11DD4
:10048000F8CF6F5F862F992783709070892B11F0BA
:100490006C7F6C5F6C5FC8010E94BB01C8010E9449
:1004A000910182E00E944401CE010E9491010E94CC
:1004B0000C0280E00E94630C8091CF048823E1F35A
:1004C000DF91CF911F910F9108950F931F93CF93B9
:1004D000DF938C01EB0160E08881882331F06F5F4E
:1004E000FE01E60FF11D8081F8CF6F5F862F9927FF
:1004F00083709070892B11F06C7F6C5F6C5FC8010A
:100500000E94BB01C8010E94910182E00E94440147
:10051000CE010E94E4010E940C0280E00E94630C64
:100520008091CF048823E1F3DF91CF911F910F9148
:100530000895EF92FF920F931F93CF93DF93CDB760
:10054000DEB728970FB6F894DEBF0FBECDBF7C0193
:1005500049835A836B837C830D831E832F83388763
:100560006CE00E94BB01C7010E94910181E00E94E2
:10057000440180E00E94AD0B6C810E94200E80E05F
:100580000E94AD0B6B810E94200E80E00E94AD0B9B
:10059000FE01319661810E94200E80E00E94AD0B29
:1005A00069810E94200E80E00E94AD0B68850E9448
:1005B000200E80E00E94AD0B6F810E94200E80E033
:1005C0000E94AD0B6E810E94200E80E00E94AD0B58
:1005D0006D810E94200E0E940C0280E00E94630C3C
:1005E0008091CF048823E1F328960FB6F894DEBFFC
:1005F0000FBECDBFDF91CF911F910F91FF90EF9074
:1006000008950F931F93CF93DF93CDB7DEB7249751
:100610000FB6F894DEBF0FBECDBF8C0149835A835D
:100620006B837C8368E00E94BB01C8010E9491013A
:1006300080E00E94440180E00E94AD0B6C810E942A
:10064000200E80E00E94AD0B6B810E94200E80E0A6
:100650000E94AD0BFE01319661810E94200E80E068
:100660000E94AD0B69810E94200E0E940C0280E066
:100670000E94630C8091CF048823E1F324960FB687
:10068000F894DEBF0FBECDBFDF91CF911F910F91C8
:1006900008950F931F938C0160E00E94BB01C80175
:1006A0000E9491010E940C0280E00E94630C8091E4
:1006B000CF048823E1F31F910F9108951092000158
:1006C0001092B4041092B2041092BA041092B904B9
:1006D00010924201109241011092B30440E450E0A4
:1006E00061E071E086EA94E00E94BD0DE1E0F1E096
:1006F0008FE31192815087FFFCCF089590934201C0
:100700008093410108950F931F93282F809100013A
:1007100099278830910509F4C6C089309105C4F441
:100720008230910509F44BC0833091052CF4009779
:1007300051F1019769F1B4C18630910509F440C1C6
:10074000873091050CF09EC1059709F451C1A8C1ED
:100750008C30910509F450C08D30910544F48A30F5
:10076000910509F4E3C00B970CF008C1B8C08E30B6
:10077000910509F46AC08E3091050CF44CC00F97B6
:1007800009F47AC08DC12E3B09F08CC181E02DC1E6
:100790002093B4041092B2042F3310F482E025C1E8
:1007A000822F9927AA27BB278C019D014FE350E098
:1007B00060E070E08CE890E00E94990244C0809173
:1007C000B204222349F0E82FFF27EF5FFE4F20837A
:1007D0008F5F8093B20466C1E82FFF27EF5FFE4F63
:1007E00020838F5F8093B204992783709070892B48
:1007F00009F058C18CE0F9C08091B204E82FFF27BE
:10080000EF5FFE4F20838F5F8093B2042C3209F09C
:1008100054C08DE0EAC08091B204E82FFF27EF5F5B
:10082000FE4F20838F5F8093B204293611F48EE04F
:10083000DCC0822F9927AA27BB27AC01BD018EE916
:1008400090E00E94010387E0D0C08091B204E82FBD
:10085000FF27EF5FFE4F20838F5F8093B204222338
:1008600011F48FE0C2C0822F9927AA27BB27AC01C1
:10087000BD018FEA90E0E5CF8091B204E82FFF2719
:10088000EF5FFE4F20838F5F8093B204222311F429
:1008900088E0ABC0822F9927AA27BB27AC01BD01F6
:1008A00080EC90E0CECF8091B204E82FFF27EF5F7D
:1008B000FE4F20838F5F8093B204822F9927AA274F
:1008C000BB27B82FAA27992788278093B504909330
:1008D000B604A093B704B093B80489E086C08091B1
:1008E000B204E82FFF27EF5FFE4F20838F5F8093D6
:1008F000B204822F9927AA27BB27AC0133272227CE
:100900008091B5049091B604A091B704B091B80459
:10091000822B932BA42BB52B8093B5049093B60414
:10092000A093B704B093B8048AE05FC08091B2048A
:10093000E82FFF27EF5FFE4F20838F5F8093B20485
:10094000822F9927AA27BB272227382F492F5A2FD2
:100950008091B5049091B604A091B704B091B80409
:10096000822B932BA42BB52B8093B5049093B604C4
:10097000A093B704B093B8048BE037C08091B20461
:10098000E82FFF27EF5FFE4F20838F5F8093B20435
:100990003327442755278091B5049091B604A09140
:1009A000B704B091B804822B932BA42BB52B809362
:1009B000B5049093B604A093B704B093B80414C0E0
:1009C0008091B204E82FFF27EF5FFE4F2083E82FCE
:1009D000EF5FE093B2048091B404E81709F062C0BD
:1009E000FF27EF5FFE4F108285E0809300015AC021
:1009F0008091B2044091B404841759F09927AA2732
:100A0000BB275527662777278C019D0181ED90E054
:100A100036C01092B30490E0941750F4392FE1E0FF
:100A2000F1E0942F8191380F9150E1F73093B304A6
:100A30008091B3048217C1F48091410190914201E9
:100A4000892B71F18091B5049091B604A091B704FF
:100A5000B091B804E0914101F0914201AC01BD01B7
:100A600081E091E009951CC09927AA27BB27422F56
:100A70005527662777278C019D0181EE90E00E9423
:100A800099020EC08091B2048F5F8093B204282F28
:100A900033278091B404992701962817390711F458
:100AA000109200011F910F9108951F93182F65E474
:100AB00080E00E94B60B612F80E00E94B60B812F70
:100AC0000E9483031F910895039665E070E00E94E1
:100AD0006413CB01AA27BB2724E0880F991FAA1F04
:100AE000BB1F2A95D1F7009711F00197FCCF08950D
:100AF0008E3040F4E82FFF27EE0FFF1FED5BFE4F17
:100B0000108211820895089593B7987F982B93BF10
:100B100008951092BB041092BC041092BD04109270
:100B2000BE041092CB041092CC041092CD0410920B
:100B3000CE04089584E00E94840512BE87B78160C8
:100B400087BF0E94890508959EB5987F982B9EBD0A
:100B5000089583E00E94A4051DBC1CBC87B7846077
:100B600087BF089595B5987F982B95BD08951092ED
:100B7000C7041092C8041092C9041092CA041092BB
:100B8000BF041092C0041092C1041092C2040895D0
:100B900082E00E94B20514BC87B7806487BF0E94C0
:100BA000B705089590918A00987F982B90938A00BA
:100BB000089583E00E94D205109289001092880067
:100BC00080917D00846080937D000895CF93C0E084
:100BD0008C2F0E947805CF5FCE30D0F30E949A050B
:100BE0000E94A9050E94C8050E94D9057894CF915A
:100BF000089583B7E82FFF27E770F070EE0FFF1F0F
:100C0000EF5FFE4F8591949108958EB5E82FFF27F1
:100C1000E770F070EE0FFF1FEF5FFE4F859194912C
:100C2000089585B5E82FFF27E770F070EE0FFF1FDE
:100C3000EF5FFE4F85919491089580918A00E82F8F
:100C4000FF27E770F070EE0FFF1FEF5FFE4F8591FB
:100C5000949108958E3040F4E82FFF27EE0FFF1F88
:100C6000ED5BFE4F6083718308950895DF92EF92EC
:100C7000FF920F931F93CF93DF93EC01D4B41092A4
:100C8000C3041092C4041092C5041092C6040E94BA
:100C900011069C014427552760E074E284EF90E040
:100CA0000E949A13293B8DE8380786E0480780E0C8
:100CB0005807C0F487E2C131D807A0F4CE01AA27B3
:100CC000BB27BC01CD010E944513DC01CB01BC0157
:100CD000CD0128EE33E040E050E00E947813FA01A5
:100CE000E90111C07E0100271127CA01B90128EED0
:100CF00033E040E050E00E947813C801B7010E9441
:100D00004513FC01EB018091C3049091C404A091B0
:100D1000C504B091C6042227382F492F5A2F84B515
:100D20009927AA27BB27282B392B4A2B5B2BCD0DC4
:100D3000D11DE11DF11D2C173D074E075F0758F52A
:100D40008091C3049091C404A091C504B091C604DD
:100D500085B7837E85BF85B7806285BF889585B757
:100D60008F7D85BF8091C3049091C404A091C50478
:100D7000B091C604BA2FA92F982F882724B53327FE
:100D800044275527822B932BA42BB52B8C179D071B
:100D9000AE07BF07A8F2DF91CF911F910F91FF908F
:100DA000EF90DF9008958091BB049091BC04A091D6
:100DB000BD04B091BE04BC01CD0108958091C7046B
:100DC0009091C804A091C904B091CA04BC01CD019E
:100DD0000895893031F48FB582608FBD8FB58E7FD5
:100DE0000AC08A3019F48FB5826002C08FB58D7F3A
:100DF0008FBD8FB581608FBD1BBC1ABC19BC18BCE0
:100E0000109279001092780008959C018FB58E7F22
:100E10008FBD8FB582608FBD8EB588608EBD8EB55B
:100E200080618EBD832F992787BD26BD1BBC1ABC50
:100E300019BC18BC109279001092780008958FB5F3
:100E40008F778FBD8FB58F7B8FBD08958FB58F7DC9
:100E50008FBD8FB58F7E8FBD08958FB5877F8FBD76
:100E60008FB58B7F8FBD08958FB58D7F8FBD8FB56B
:100E70008E7F8FBD0E941F070E9426070E942D07AC
:100E800008958FB580688FBD8FB58F7B8FBD089516
:100E90008FB580628FBD8FB58F7E8FBD08958FB562
:100EA00088608FBD8FB58B7F8FBD08959C01892F82
:100EB00099278BBD2ABD08959C01892F992789BD4B
:100EC00028BD08959C01892F99278093790020934C
:100ED00078000895893049F480918B008260809376
:100EE0008B0080918B008E7F0EC08A3021F4809120
:100EF0008B00826003C080918B008D7F80938B007C
:100F000080918B00816080938B00109287001092FB
:100F10008600109285001092840010928300109237
:100F2000820008959C0180918B008E7F80938B00BE
:100F300080918B00826080938B0080918A00886012
:100F400080938A0080918A00806180938A00832F39
:100F5000992780938100209380001092870010923F
:100F600086001092850010928400109283001092E7
:100F70008200089580918B008F7780938B00809101
:100F80008B008F7B80938B00089580918B008F7DE9
:100F900080938B0080918B008F7E80938B000895CF
:100FA00080918B00877F80938B0080918B008B7F5B
:100FB00080938B00089580918B008D7F80938B00B0
:100FC00080918B008E7F80938B000E94BA070E94D5
:100FD000C5070E94D007089580918B008068809398
:100FE0008B0080918B008F7B80938B000895809184
:100FF0008B00806280938B0080918B008F7E80932A
:101000008B00089580918B00886080938B00809185
:101010008B008B7F80938B0008959C01892F9927EB
:10102000809387002093860008959C01892F99273B
:10103000809385002093840008959C01832F992735
:10104000809383002093820008951F920F920FB621
:101050000F9211242F933F934F935F936F937F933E
:101060008F939F93AF93BF93EF93FF938091BB04B4
:101070009091BC04A091BD04B091BE040196A11D45
:10108000B11D8093BB049093BC04A093BD04B093A6
:10109000BE048091BB049091BC04A091BD04B091AA
:1010A000BE040097A105B10599F48091CB049091FD
:1010B000CC04A091CD04B091CE040196A11DB11D28
:1010C0008093CB049093CC04A093CD04B093CE0432
:1010D0008091430190914401892B29F0E0914301D3
:1010E000F09144010995FF91EF91BF91AF919F91CC
:1010F0008F917F916F915F914F913F912F910F90C1
:101100000FBE0F901F9018951F920F920FB60F925F
:1011100011242F933F934F935F936F937F938F93FC
:101120009F93AF93BF93EF93FF938091470190916B
:101130004801892B29F0E0914701F0914801099578
:10114000FF91EF91BF91AF919F918F917F916F919F
:101150005F914F913F912F910F900FBE0F901F9075
:1011600018951F920F920FB60F9211242F933F9351
:101170004F935F936F937F938F939F93AF93BF939F
:10118000EF93FF938091C7049091C804A091C90484
:10119000B091CA040196A11DB11D8093C70490931C
:1011A000C804A093C904B093CA048091C704909165
:1011B000C804A091C904B091CA040097A105B10563
:1011C00099F48091BF049091C004A091C104B091A2
:1011D000C2040196A11DB11D8093BF049093C00469
:1011E000A093C104B093C2048091C3049091C4043D
:1011F000A091C504B091C6040196A11DB11D8093B4
:10120000C3049093C404A093C504B093C604809112
:10121000510190915201892B29F0E0915101F091F7
:1012200052010995FF91EF91BF91AF919F918F91DD
:101230007F916F915F914F913F912F910F900FBED2
:101240000F901F9018951F920F920FB60F921124B6
:101250002F933F934F935F936F937F938F939F93BE
:10126000AF93BF93EF93FF938091550190915601F7
:10127000892B29F0E0915501F09156010995FF91D4
:10128000EF91BF91AF919F918F917F916F915F91FE
:101290004F913F912F910F900FBE0F901F90189577
:1012A0001F920F920FB60F9211242F933F934F93DB
:1012B0005F936F937F938F939F93AF93BF93EF93BE
:1012C000FF938091450190914601892B29F0E0918F
:1012D0004501F09146010995FF91EF91BF91AF91C2
:1012E0009F918F917F916F915F914F913F912F913E
:1012F0000F900FBE0F901F9018951F920F920FB670
:101300000F9211242F933F934F935F936F937F938B
:101310008F939F93AF93BF93EF93FF938091490176
:1013200090914A01892B29F0E0914901F0914A01FD
:101330000995FF91EF91BF91AF919F918F917F910F
:101340006F915F914F913F912F910F900FBE0F9032
:101350001F9018951F920F920FB60F9211242F9382
:101360003F934F935F936F937F938F939F93AF932D
:10137000BF93EF93FF9380914B0190914C01892B88
:1013800029F0E0914B01F0914C010995FF91EF910B
:10139000BF91AF919F918F917F916F915F914F918D
:1013A0003F912F910F900FBE0F901F9018951F9295
:1013B0000F920FB60F9211242F933F934F935F9389
:1013C0006F937F938F939F93AF93BF93EF93FF930D
:1013D00080914D0190914E01892B29F0E0914D01B2
:1013E000F0914E010995FF91EF91BF91AF919F91BF
:1013F0008F917F916F915F914F913F912F910F90BE
:101400000FBE0F901F9018951F920F920FB60F925C
:1014100011242F933F934F935F936F937F938F93F9
:101420009F93AF93BF93EF93FF9380914F01909160
:101430005001892B29F0E0914F01F091500109955D
:10144000FF91EF91BF91AF919F918F917F916F919C
:101450005F914F913F912F910F900FBE0F901F9072
:1014600018951F920F920FB60F9211242F933F934E
:101470004F935F936F937F938F939F93AF93BF939C
:10148000EF93FF938091530190915401892B29F0A0
:10149000E0915301F09154010995FF91EF91BF91B3
:1014A000AF919F918F917F916F915F914F913F91FC
:1014B0002F910F900FBE0F901F9018951F920F92B3
:1014C0000FB60F9211242F933F934F935F936F9317
:1014D0007F938F939F93AF93BF93EF93FF938091ED
:1014E000570190915801892B29F0E0915701F09113
:1014F00058010995FF91EF91BF91AF919F918F9105
:101500007F916F915F914F913F912F910F900FBEFF
:101510000F901F9018951F920F920FB60F921124E3
:101520002F933F934F935F936F937F938F939F93EB
:10153000AF93BF93EF93FF938091590190915A011C
:10154000892B29F0E0915901F0915A010995FF91F9
:10155000EF91BF91AF919F918F917F916F915F912B
:101560004F913F912F910F900FBE0F901F901895A4
:101570001F920F920FB60F9211242F933F934F9308
:101580005F936F937F938F939F93AF93BF93EF93EB
:10159000FF9380915B0190915C01892B29F0E09190
:1015A0005B01F0915C010995FF91EF91BF91AF91C3
:1015B0009F918F917F916F915F914F913F912F916B
:1015C0000F900FBE0F901F9018951F920F920FB69D
:1015D0000F9211242F933F934F935F936F937F93B9
:1015E0008F939F93AF93BF93EF93FF9380915D0190
:1015F00090915E01892B29F0E0915D01F0915E01EF
:101600000995FF91EF91BF91AF919F918F917F913C
:101610006F915F914F913F912F910F900FBE0F905F
:101620001F9018951F93182FDB01CA0173E0880FD4
:10163000991FAA1FBB1F7A95D1F79C01AD01220FFC
:10164000331F441F551F80509C4DAB40BF4FBC0102
:10165000CD010E947813DA01C9010197292F3327A0
:10166000112329F0809399002093980003C089B931
:10167000209390001F91089540E250E06FE574E0E0
:1016800089ED94E00E94BD0D40E250E06FE774E008
:101690008BEE94E00E94BD0D08950E943C0B1092C9
:1016A000A2041092A10488ED80939A0040E855E2CC
:1016B00060E070E081E00E94120B8FEF8093D00415
:1016C0001092E2041092F6041092F50478940895B2
:1016D00040E052E06FE571E081ED94E00E94BD0DC5
:1016E00040E051E06FE573E083EE94E00E94BD0DB1
:1016F00008950E94680B1092A00410929F0488ED38
:101700008AB940E855E260E070E080E00E94120B88
:101710008FEF8093CF041092E1041092F4041092A2
:10172000F304789408950E94790B0E944D0B08955C
:10173000823040F4E82FFF27EE0FFF1FE156FB4FEA
:1017400060837183089508959927E3E0880F991FB6
:10175000EA95E1F78F529B4F08959927F3E0880FA0
:10176000991FFA95E1F78D519B4F0895982FE82F17
:10177000FF27DF01A153BB4F8C918823E9F3992305
:1017800019F060939C0001C06CB9E153FB4F1082CB
:101790000895682F80E00E94B60B0895682F81E0BD
:1017A0000E94B60B0895CF93DF93EB01E82FFF273C
:1017B000A3E0EE0FFF1FAA95E1F7EF52FB4F8281E6
:1017C0009381009751F084819581009731F0CF018A
:1017D0000E94C70D88838FEF90E0DF91CF9108952D
:1017E000CF93DF93CDB7DEB721970FB6F894DEBF66
:1017F0000FBECDBFBE016F5F7F4F81E00E94D30B54
:10180000882319F08981992702C08FEF9FEF2196D5
:101810000FB6F894DEBF0FBECDBFDF91CF91089514
:10182000CF93DF93CDB7DEB721970FB6F894DEBF25
:101830000FBECDBFBE016F5F7F4F80E00E94D30B14
:10184000882319F08981992702C08FEF9FEF219695
:101850000FB6F894DEBF0FBECDBFDF91CF910895D4
:101860009927B3E0880F991FBA95E1F78F529B4FE4
:101870000E94510E089520E030E0E82FFF2783E01A
:10188000EE0FFF1F8A95E1F7EF52FB4F84819581A0
:10189000892B11F421E030E0C9010895992733E044
:1018A000880F991F3A95E1F78D519B4F0E94200EAA
:1018B0000895682F80E00E944E0C0895682F81E003
:1018C0000E944E0C08951F93182F9927FC01EF5189
:1018D000FB4F2FEF208343E0880F991F4A95E1F7D4
:1018E0008D519B4F0E94C70D682F812F0E94B60B10
:1018F0001F910895CF92DF92EF92FF920F931F9363
:10190000CF93DF93D82E8B01E82EFF24F70163E0FD
:10191000EE0FFF1F6A95E1F7ED51FB4F8481958132
:10192000840F951F228133818217930740F541155B
:10193000510529F1F801C1908F014130510591F015
:10194000EA012197F80121918F01C70153E0880F27
:10195000991F5A95E1F7622F8D519B4F0E94200EDF
:10196000219781F7ED2DFF27EF51FB4F8FEF8083FC
:101970006C2D8D2D0E94B60B8FEF90E002C080E0A1
:1019800090E0DF91CF911F910F91FF90EF90DF904A
:10199000CF900895CF93DF93282FA82FBB27ED0179
:1019A000CF51DB4F88818823E1F0FD0173E0EE0F1A
:1019B000FF1F7A95E1F7ED51FB4F84819581892BCB
:1019C00079F0222339F08BEE94E00E94C70D8093CA
:1019D0009C000BC083EE94E00E94C70D8CB905C03B
:1019E0001882A153BB4F8FEF8C93DF91CF91089555
:1019F000CF93DF93882319F060919C0001C06CB1F4
:101A0000282F3327E901C20FD31FFE01E156FB4FF8
:101A100080819181892B31F00190F081E02D862F1A
:101A2000099514C0E3E0220F331FEA95E1F7C901DD
:101A30008F529B4F0E94200E882341F4FE01ED50EF
:101A4000FB4F80819181019680839183DF91CF91BB
:101A500008951F920F920FB60F9211242F933F9368
:101A60004F935F936F937F938F939F93AF93BF93A6
:101A7000EF93FF9380E00E94CA0CFF91EF91BF911A
:101A8000AF919F918F917F916F915F914F913F9116
:101A90002F910F900FBE0F901F9018951F920F92CD
:101AA0000FB60F9211242F933F934F935F936F9331
:101AB0007F938F939F93AF93BF93EF93FF9381E0B7
:101AC0000E94CA0CFF91EF91BF91AF919F918F91AE
:101AD0007F916F915F914F913F912F910F900FBE2A
:101AE0000F901F9018951F920F920FB60F9211240E
:101AF0002F933F934F935F936F937F938F939F9316
:101B0000AF93BF93EF93FF9380E00E94F80CFF9197
:101B1000EF91BF91AF919F918F917F916F915F9165
:101B20004F913F912F910F900FBE0F901F901895DE
:101B30001F920F920FB60F9211242F933F934F9342
:101B40005F936F937F938F939F93AF93BF93EF9325
:101B5000FF9381E00E94F80CFF91EF91BF91AF914C
:101B60009F918F917F916F915F914F913F912F91B5
:101B70000F900FBE0F901F901895FC01608371832A
:101B80004283538316821782148215820895CF935D
:101B9000DF93EC01E0E02C813D8121153105B9F0A6
:101BA0008E819F81E881F981E80FF91FE08101961C
:101BB0008E839F836A817B818617970720F00E941E
:101BC00064138E839F83215030402C833D838E2F5E
:101BD0009927DF91CF910895CF93DF93FC01EB011B
:101BE0002481358162177307A0F486819781860F5F
:101BF000971F86839783628173818617970720F0EA
:101C00000E946413868397832C1B3D0B24833583AA
:101C100002C014821582DF91CF910895FC01868164
:101C2000978122813381860F971FB9010E94641327
:101C30000190F081E02DE80FF91F80819927089528
:101C4000CF93DF93EC01462F2C813D816A817B810C
:101C50002617370798F48E819F81820F931F0E9469
:101C60006413E881F981E80FF91F40838C819D811D
:101C700001968C839D838FEF90E002C080E090E01E
:101C8000DF91CF910895FC0140E050E0248135813F
:101C9000828193812817390710F441E050E0CA018E
:101CA0000895FC011482158208959093A4048093F2
:101CB000A3040895E091A304F091A4040995089564
:101CC000CF93DF93EC01892B61F08881882349F061
:101CD000E091A304F091A404899109958881882357
:101CE000B9F7DF91CF910895EF92FF920F931F9371
:101CF000CF93DF93EC017A0120E030E0892B01F1F2
:101D0000C9012F5F3F4F8617970718F489918823E1
:101D1000B9F720E030E02E153F0590F48881890165
:101D20000F5F1F4FE091A304F091A404882311F0EA
:101D3000219601C080E2099598010E151F0570F3E8
:101D4000DF91CF911F910F91FF90EF900895CF9366
:101D5000DF93EC01009779F0FC01219684918823B0
:101D600051F0E091A304F091A4040995FE0121969D
:101D700084918823B1F7DF91CF910895E091A30476
:101D8000F091A4048DE00995E091A304F091A404DE
:101D90008AE009950895E82FFF27EF70F070E35F60
:101DA000FE4F8491E091A304F091A4040995089555
:101DB0001F93182F82958F700E94CB0E812F0E9447
:101DC000CB0E1F9108950F931F938C01812F99279C
:101DD0000E94D80E802F0E94D80E1F910F91089557
:101DE000EF92FF920F931F937B018C01C801AA27EA
:101DF000BB270E94E30EC7010E94E30E1F910F91C3
:101E0000FF90EF9008952F923F924F925F926F92C2
:101E10007F928F929F92AF92BF92CF92DF92EF927A
:101E2000FF920F931F93CF93DF93CDB7DEB7A297A7
:101E30000FB6F894DEBF0FBECDBF69A3C42E2AA390
:101E400027013801442351F017FF08C0EE24FF2476
:101E50008701E418F5080609170902C08301720119
:101E600099A1692F772767FD709561507040CC204C
:101E700011F061507040D62E18A22FE1222E312C85
:101E80002C0E3D1E882E992487FC9094A92CB92CE9
:101E9000C801B701A50194010E947813DC01CB01B0
:101EA000FC01E35FFE4F84918F8FC801B701A5014C
:101EB00094010E94781379018A01DA94AFEFDA165F
:101EC00039F1DA94C1010197E114F104010511051A
:101ED000C1F01C01C801B701A50194010E9478134B
:101EE000DC01CB01FC01E35FFE4F8491F1018083B3
:101EF000C801B701A50194010E94781379018A01F4
:101F000004C01C01EAA1DC01EC93FFEFDF16C9F667
:101F1000CC20B9F077FE05C08DE2D1018E931D0172
:101F200010C0C101019714141504160417042CF4F1
:101F30001C018BE2F101808304C01C0180E2D1010D
:101F40008C93D9A0DA94BFEFDB1661F0E091A30483
:101F5000F091A404D1018D911D010995DA94BFEF90
:101F6000DB16A1F7A2960FB6F894DEBF0FBECDBF69
:101F7000DF91CF911F910F91FF90EF90DF90CF9065
:101F8000BF90AF909F908F907F906F905F904F9099
:101F90003F902F9008957F928F929F92AF92BF9221
:101FA000CF92DF92EF92FF920F931F93CF93DF9325
:101FB000CDB7DEB77888C988DA8863E1A62EB12C60
:101FC000AC0EBD1E08C0882309F481C0E091A304B3
:101FD000F091A404099596012F5F3F4F772021F0DF
:101FE000F6016901849103C0F6018081690185329F
:101FF00051F72F5F3F4F772021F0F601690184915F
:1020000003C0F60180816901282F332727FD309511
:102010002436310591F02536310524F42336310577
:1020200029F0D4CF2837310581F0D0CFF50122E057
:1020300030E0A20EB31E8081C9CF5AE0852E912CCC
:1020400040E1E42E47E2F42E04C030E1E32EF12C0F
:102050004701F50122E030E0A20EB31E008111819C
:102060008436D9F417FF09C0109501951F4FE091F0
:10207000A304F091A4048DE2099532E0E316F10483
:1020800060F00E151F0548F4C7016AE070E00E9479
:1020900064137B0162307105A0F7C801B7010E948B
:1020A0006413FB01E35FFE4F8491E091A304F09180
:1020B000A4040995C801B7010E9464138C01C701EB
:1020C000B4010E9464137B01672B39F784CF80E051
:1020D00090E0DF91CF911F910F91FF90EF90DF90F3
:1020E000CF90BF90AF909F908F907F9008958091F8
:1020F000650081608093650085E090E00E9436066F
:10210000809165008E7F809365000895CEEFD0E1C9
:10211000DEBFCDBF0E94E60580E00E94771081E01F
:10212000809364001092650014BA8FEF85BB8ABB60
:102130001BBA0E94EF00BD9ABE9ABF9A139A149AD6
:10214000159A0E94A90588E00E94E9060E944107AD
:102150000E9448070E944F0780E090E00E945607C7
:1021600080E090E00E945C0780E090E00E946207BF
:102170000E94D90588E00E946A070E94EC070E942D
:10218000F7070E94020880E090E00E940D0880E0BE
:1021900090E00E94150880E090E00E941D080E94D7
:1021A000790B40E052EC61E070E080E00E94120B9D
:1021B0000E943A010E945E038EEF90E10E947E032E
:1021C00001E010E0BE016F5F7F4F80E00E94D30B03
:1021D000882319F089810E948303C801817090705F
:1021E0000F5F1F4F892B21F080916500816003C034
:1021F000809165008E7F80936500E4CFDF92EF923F
:10220000FF920F931F93CF93DF93EC017A018B0121
:10221000DD2444E050E06EE171E00E943713892B29
:10222000A9F5FE0101900020E9F73697EC17FD07AC
:1022300009F095C08C81803329F48E2D99270E9456
:102240001D088DC0813329F48E2D99270E94150811
:1022500086C0823329F48E2D99270E940D087FC0F5
:10226000833329F48E2D99270E94620778C0843326
:1022700029F48E2D99270E945C0771C0853309F0DF
:102280006EC08E2D99270E94560769C044E050E029
:1022900063E271E0CE010E943713892B09F05FC021
:1022A000FE0101900020E9F73697EC17FD0709F0D1
:1022B00056C08C81992787FD909583339105F1F065
:1022C000843391054CF48133910591F0823391056B
:1022D00094F4C09709F143C085339105A9F0853383
:1022E00091057CF08633910591F0C79799F037C03E
:1022F00061E0D62E11C052E0D52E0EC043E0D42EA0
:102300000BC034E0D32E08C025E0D22E05C096E0E5
:10231000D92E02C087E0D82E81E090E0A0E0B0E0A6
:10232000E822F9220A231B232D2D3327EF2869F0F9
:1023300081E090E002C0880F991F2A95E2F7982F5C
:1023400090958BB389238BBB0AC081E090E002C0DB
:10235000880F991F2A95E2F72BB3282B2BBBDF910F
:10236000CF911F910F91FF90EF90DF9008951F93F1
:10237000CF93DF9313B3C12FDD279E0121703070FF
:10238000809107059927817090702817390781F08F
:1023900081E090E08C279D27AA27BB278170907051
:1023A000A070B070AC01BD0188E291E00E94010311
:1023B0009E0122703070809107059927827090707D
:1023C0002817390799F0CE019695879521E030E0DE
:1023D00082279327AA27BB2781709070A070B070C6
:1023E000AC01BD018DE291E00E9401039E012470C9
:1023F00030708091070599278470907028173907ED
:10240000A9F0CE01969587959695879521E030E0C5
:1024100082279327AA27BB2781709070A070B07085
:10242000AC01BD0182E391E00E9401039E0128708E
:1024300030708091070599278870907028173907A8
:10244000B1F0CE01B3E096958795BA95E1F721E01A
:1024500030E082279327AA27BB2781709070A07055
:10246000B070AC01BD0187E391E00E9401039E01C1
:10247000207130708091070599278071907028171E
:102480003907B1F0CE01A4E096958795AA95E1F7BA
:1024900021E030E082279327AA27BB278170907024
:1024A000A070B070AC01BD018CE391E00E9401030B
:1024B0009E0120723070809107059927807290707C
:1024C00028173907B1F0CE01F5E096958795FA9572
:1024D000E1F721E030E082279327AA27BB2781700C
:1024E0009070A070B070AC01BD0181E491E00E94D9
:1024F00001039E0120743070809107059927807434
:10250000907028173907B1F0CE01E6E096958795CF
:10251000EA95E1F721E030E082279327AA27BB273D
:1025200081709070A070B070AC01BD0186E491E044
:102530000E940103C078D0708091070599278078A8
:102540009070C817D907B1F0812F992787FD909512
:10255000A92FB92F80959095A095B0958827B7FDA4
:1025600083959927AA27BB27AC01BD018BE491E095
:102570000E94010310930705DF91CF911F910895E9
:102580001F93182F0E940E01AC01212F3327F90150
:10259000E20FF31FE950FB4F80819181BA01681B64
:1025A000790BCB010896419708F45FC040835183B3
:1025B0002330310589F1243031054CF421303105C7
:1025C000D9F02230310504F5232B71F04EC02530AF
:1025D000310591F1253031053CF126303105A1F16D
:1025E00027303105C9F141C0CA01AA27BB27AC0178
:1025F000BD0180E591E037C0CA01AA27BB27AC0125
:10260000BD0186E591E02FC0CA01AA27BB27AC0116
:10261000BD018CE591E027C0CA01AA27BB27AC0108
:10262000BD0182E691E01FC0CA01AA27BB27AC0109
:10263000BD0188E691E017C0CA01AA27BB27AC01FB
:10264000BD018EE691E00FC0CA01AA27BB27AC01ED
:10265000BD0184E791E007C0CA01AA27BB27AC01EE
:10266000BD018AE791E00E9401031F910895FB01DB
:10267000DC014150504030F08D910590801919F4E3
:102680000020B9F7881B990B0895629FD001739FB2
:10269000F001829FE00DF11D649FE00DF11D929FFE
:1026A000F00D839FF00D749FF00D659FF00D99273D
:1026B000729FB00DE11DF91F639FB00DE11DF91F61
:1026C000BD01CF0111240895AA1BBB1B51E107C016
:1026D000AA1FBB1FA617B70710F0A61BB70B881FB2
:1026E000991F5A95A9F780959095BC01CD01089541
:1026F000A1E21A2EAA1BBB1BFD010DC0AA1FBB1F06
:10270000EE1FFF1FA217B307E407F50720F0A21B77
:10271000B30BE40BF50B661F771F881F991F1A94E4
:1027200069F760957095809590959B01AC01BD010E
:10273000CF01089597FB092E05260ED057FD04D032
:10274000D7DF0AD0001C38F450954095309521957C
:102750003F4F4F4F5F4F0895F6F7909580957095D6
:0A27600061957F4F8F4F9F4F089542
:00000001FF
